:020000020000FC
:0200000020C01E
:0200280054C0C2
:100040002DC000E00ABB00E00BBB0FEF07BB0FEFBA
:1000500008BB0FEF04BB0FEF05BB0FEF01BB0FEFAA
:1000600002BB0FE50DBF08E00EBF61E00CE003BF6F
:1000700006E20CBF02E009BF00EC07B900E808B9CE
:100080000BE006B900E805BF78948895F9CF0BE836
:1000900006B900E905BF78948895089504B115B1B3
:1000A00020E030E040E0043618F4113008F404C0D9
:1000B000045610404395F7CF4A3038F40A3018F010
:1000C0000A503395FBCF202F03C02FEF3FEF4FEFA8
:1000D000189506D053956A9511F469E1D8DF189503
:1000E000042F10D0006850FD009502BB032F0AD0EA
:1000F0000F7750FD009505BB022F04D050FD0095F1
:1001000008BB08950030A1F00130A1F00230A1F049
:100110000330A1F00430A1F00530A1F00630A1F0C9
:100120000730A1F00830A1F00930A1F00FEB0895DD
:1001300000EC089509EF089504EA089500EB08958E
:1001400009E9089502E9089502E8089508EF08957D
:0801500000E8089500E908959C
:00000001FF
